:020000040801F1
:1000000000000220B9260108551101085911010804
:100010005D1101086111010865110108000000006F
:10002000000000000000000000000000691101084D
:100030006D1101080000000071110108751101081F
:1000400009270108092701080927010809270108CC
:1000500009270108092701080927010809270108BC
:1000600009270108092701080927010809270108AC
:10007000092701080927010809270108092701089C
:10008000092701080927010809270108092701088C
:10009000092701080927010809270108092701087C
:1000A000092701080927010809270108092701086C
:1000B000092701080927010809270108092701085C
:1000C000092701080927010809270108092701084C
:1000D0000927010885110108911101080927010864
:1000E000092701080927010809270108092701082C
:1000F000092701080927010809270108092701081C
:10010000092701080927010809270108092701080B
:100110009D1101080927010809270108092701087D
:1001200009270108092701080927010809270108EB
:1001300009270108092701080927010809270108DB
:1001400009270108092701080927010809270108CB
:1001500009270108092701080927010809270108BB
:1001600009270108092701080927010809270108AB
:1001700009270108092701080927010800000000D4
:08018000092701080927010805
:10018800044B05481B1A062B02D9044B03B1184728
:10019800704700BF1300002010000020000000007E
:1001A80005490648091A891001EBD171491002D096
:1001B800034B03B1184770471000002010000020BF
:1001C8000000000010B5064C237843B9FFF7D8FFAC
:1001D800044B13B10448AFF300800123237010BD12
:1001E80010000020000000000C27010808B5084B8B
:1001F8001BB108490848AFF300800848036813B9E1
:10020800BDE80840CCE7064B002BF9D09847F7E744
:1002180000000000140000200C2701081000002036
:100228000000000070B50F4E0F4D761BB61018BFBA
:10023800002405D0013455F8043B9847A642F9D16B
:100248000A4E0B4D761B02F05DFAB61018BF00245B
:1002580006D0013455F8043B9847A642F9D170BD41
:1002680070BD00BF3427010834270108382701086A
:100278003427010870B4860746D0541E002A41D09E
:10028800CAB2034602E014F1FF343BD303F8012B52
:100298009D07F8D1032C2ED9CDB245EA05250F2CA0
:1002A80045EA054519D903F110022646103E0F2EDE
:1002B80042F8105C42F80C5C42F8085C42F8045CB6
:1002C80002F11002F2D8A4F1100222F00F0204F099
:1002D8000F041032032C13440DD91E462246043A4B
:1002E800032A46F8045BFAD8221F22F003020432DC
:1002F800134404F003042CB1C9B21C4403F8011BD5
:100308009C42FBD170BC704714460346C2E700BF4D
:1003180081F0004102E000BF83F0004330B54FEAAE
:1003280041044FEA430594EA050F08BF90EA020F1B
:100338001FBF54EA000C55EA020C7FEA645C7FEAAE
:10034800655C00F0E2804FEA5454D4EB5555B8BFD1
:100358006D420CDD2C4480EA020281EA030382EA42
:10036800000083EA010180EA020281EA0303362DD4
:1003780088BF30BD11F0004F4FEA01314FF4801CA7
:100388004CEA113102D0404261EB410113F0004FB9
:100398004FEA03334CEA133302D0524263EB430370
:1003A80094EA050F00F0A780A4F10104D5F1200E0E
:1003B8000DDB02FA0EFC22FA05F2801841F1000169
:1003C80003FA0EF2801843FA05F359410EE0A5F13D
:1003D80020050EF1200E012A03FA0EFC28BF4CF06E
:1003E800020C43FA05F3C01851EBE37101F0004524
:1003F80007D54FF0000EDCF1000C7EEB00006EEB31
:100408000101B1F5801F1BD3B1F5001F0CD34908BA
:100418005FEA30004FEA3C0C04F101044FEA445211
:1004280012F5800F80F09A80BCF1004F08BF5FEA98
:10043800500C50F1000041EB045141EA050130BD78
:100448005FEA4C0C404141EB010111F4801FA4F11B
:100458000104E9D191F0000F04BF01460020B1FA70
:1004680081F308BF2033A3F10B03B3F120020CDAA8
:100478000C3208DD02F1140CC2F10C0201FA0CF086
:1004880021FA02F10CE002F11402D8BFC2F1200CEB
:1004980001FA02F120FA0CFCDCBF41EA0C019040A1
:1004A800E41AA2BF01EB0451294330BD6FEA0404EA
:1004B8001F3C1CDA0C340EDC04F11404C4F12002D5
:1004C80020FA04F001FA02F340EA030021FA04F3E7
:1004D80045EA030130BDC4F10C04C4F1200220FA3E
:1004E80002F001FA04F340EA0300294630BD21FA7C
:1004F80004F0294630BD94F0000F83F4801306BF42
:1005080081F480110134013D4EE77FEA645C18BF35
:100518007FEA655C29D094EA050F08BF90EA020FCC
:1005280005D054EA000C04BF1946104630BD91EAC4
:10053800030F1EBF0021002030BD5FEA545C05D1C7
:100548004000494128BF41F0004130BD14F5800406
:100558003CBF01F5801130BD01F0004545F0FE417A
:1005680041F470014FF0000030BD7FEA645C1ABFAF
:10057800194610467FEA655C1CBF0B46024650EAE6
:10058800013406BF52EA033591EA030F41F4002112
:1005980030BD00BF90F0000F04BF0021704730B598
:1005A8004FF4806404F132044FF000054FF000016D
:1005B80050E700BF90F0000F04BF0021704730B52E
:1005C8004FF4806404F1320410F0004548BF404203
:1005D8004FF000013EE700BF42004FEAE2014FEA58
:1005E80031014FEA02701FBF12F07F4393F07F4F33
:1005F80081F06051704792F0000F14BF93F07F4F65
:10060800704730B54FF4607401F0004521F00041A7
:1006180020E700BF50EA010208BF704730B54FF02D
:1006280000050AE050EA010208BF704730B511F032
:10063800004502D5404261EB41014FF4806404F16A
:1006480032045FEA915C3FF4DCAE4FF003025FEAEC
:10065800DC0C18BF03325FEADC0C18BF033202EB74
:10066800DC02C2F1200300FA03FC20FA02F001FACE
:1006780003FE40EA0E0021FA02F11444C1E600BF6D
:1006880070B54FF0FF0C4CF4E06C1CEA11541DBF20
:100698001CEA135594EA0C0F95EA0C0F00F0DEF8EB
:1006A8002C4481EA030621EA4C5123EA4C5350EAD0
:1006B800013518BF52EA033541F4801143F4801321
:1006C80038D0A0FB02CE4FF00005E1FB02E506F0B2
:1006D8000042E0FB03E54FF00006E1FB03569CF007
:1006E800000F18BF4EF0010EA4F1FF04B6F5007F0D
:1006F80064F5407404D25FEA4E0E6D4146EB06067F
:1007080042EAC62141EA55514FEAC52040EA5E5007
:100718004FEACE2EB4F1FD0C88BFBCF5E06F1ED8B1
:10072800BEF1004F08BF5FEA500E50F1000041EBE8
:10073800045170BD06F0004646EA010140EA020095
:1007480081EA0301B4EB5C04C2BFD4EB0C0541EAB7
:10075800045170BD41F480114FF0000E013C00F3CC
:10076800AB8014F1360FDEBF002001F0004170BDF0
:10077800C4F10004203C35DA0C341BDC04F1140409
:10078800C4F1200500FA05F320FA04F001FA05F295
:1007980040EA020001F0004221F0004110EBD37062
:1007A80021FA04F642EB06015EEA430E08BF20EA8E
:1007B800D37070BDC4F10C04C4F1200500FA04F331
:1007C80020FA05F001FA04F240EA020001F00041C3
:1007D80010EBD37041F100015EEA430E08BF20EA36
:1007E800D37070BDC4F1200500FA05F24EEA020E7E
:1007F80020FA04F301FA05F243EA020321FA04F0AD
:1008080001F0004121FA04F220EA020000EBD37063
:100818005EEA430E08BF20EAD37070BD94F0000F63
:100828000FD101F00046400041EB010111F4801F97
:1008380008BF013CF7D041EA060195F0000F18BF48
:10084800704703F00046520043EB030313F4801F84
:1008580008BF013DF7D043EA0603704794EA0C0F3E
:100868000CEA135518BF95EA0C0F0CD050EA410654
:1008780018BF52EA4306D1D181EA030101F00041D1
:100888004FF0000070BD50EA410606BF10461946F9
:1008980052EA430619D094EA0C0F02D150EA013605
:1008A80013D195EA0C0F05D152EA03361CBF104646
:1008B80019460AD181EA030101F0004141F0FE41E5
:1008C80041F470014FF0000070BD41F0FE4141F469
:1008D800780170BD70B54FF0FF0C4CF4E06C1CEA69
:1008E80011541DBF1CEA135594EA0C0F95EA0C0F1E
:1008F80000F0A7F8A4EB050481EA030E52EA0335D9
:100908004FEA013100F088804FEA03334FF08055F9
:1009180045EA131343EA12634FEA022245EA111526
:1009280045EA10654FEA00260EF000419D4208BFD7
:10093800964244F1FD0404F5407402D25B084FEA84
:100948003202B61A65EB03055B084FEA32024FF430
:1009580080104FF4002CB6EB020E75EB030E22BF8D
:10096800B61A754640EA0C005B084FEA3202B6EB4D
:10097800020E75EB030E22BFB61A754640EA5C00FC
:100988005B084FEA3202B6EB020E75EB030E22BF8C
:10099800B61A754640EA9C005B084FEA3202B6EB8D
:1009A800020E75EB030E22BFB61A754640EADC004C
:1009B80055EA060E18D04FEA051545EA16754FEAAE
:1009C80006164FEAC30343EA52734FEAC2025FEACC
:1009D8001C1CC0D111F4801F0BD141EA00014FF05B
:1009E80000004FF0004CB6E711F4801F04BF01432C
:1009F8000020B4F1FD0C88BFBCF5E06F3FF6AFAE48
:100A0800B5EB030C04BFB6EB020C5FEA500C50F1D7
:100A1800000041EB045170BD0EF0004E4EEA11315A
:100A280014EB5C04C2BFD4EB0C0541EA045170BD61
:100A380041F480114FF0000E013C90E645EA060EA5
:100A48008DE60CEA135594EA0C0F08BF95EA0C0FD3
:100A58003FF43BAF94EA0C0F0AD150EA01347FF41B
:100A680034AF95EA0C0F7FF425AF104619462CE7F2
:100A780095EA0C0F06D152EA03353FF4FDAE104655
:100A8800194622E750EA410618BF52EA43067FF4A6
:100A9800C5AE50EA41047FF40DAF52EA43057FF436
:100AA800EBAE12E74FEA4102B2F1E04324BFB3F5DF
:100AB800001CDCF1FE5C0DD901F0004C4FEAC002CD
:100AC8004CEA5070B2F1004F40EB830008BF20F0B1
:100AD8000100704711F0804F21D113F13872BCBF6B
:100AE80001F00040704741F480114FEA5252C2F1C0
:100AF8001802C2F1200C10FA0CF320FA02F018BF09
:100B080040F001004FEAC1234FEAD32303FA0CFC5B
:100B180040EA0C0023FA02F34FEA4303CCE77FEAEA
:100B2800625307D150EA01331EBF4FF0FE4040F434
:100B38004000704701F0004040F0FE4040F40000E3
:100B4800704700BFF0B595B008A830220021FFF724
:100B580091FB00241D4A019404940394059406947F
:100B68000794116C1A4B41F080511164126C02F019
:100B780080520192019A02941A6842F480421A60E3
:100B88001B680F9403F48043029301230225082174
:100B980048220B9308A8032310261091119213934F
:100BA800029F08950E9512950C9601F08FF80F226A
:100BB8004FF4805303A8294604950594079403929B
:100BC800069301F079FA15B0F0BD00BF0038024075
:100BD80000700040F0B5114C114A124B226085B0EC
:100BE8000025012607462046A36265600095A5609A
:100BF8002561A5612562E562E56025630195029599
:100C08000395E661666100F0FBFA694620460097A5
:100C18000196029500F068FC05B0F0BD3800002090
:100C2800002001400100000FD0B500202DED028BFF
:100C3800FFF7D0FF324800F097FB3221304800F030
:100C4800FFFB2F4800F0F4FC83050DD40A2304228F
:100C58002C492D4800F0CAFEBDEC028B42F2107000
:100C6800BDE8D04001F0EEBC254800F039FC83B265
:100C780008EE103A9FED257ADFED257A2549264AB8
:100C8800D1ED008A254B1080B8EEC88A28EE078A75
:100C980028EE278AB4EEE88AF1EE10FA83ED008A8E
:100CA80027DC1F4B174CD3ED007A78EEE77A17EE66
:100CB800900AFFF791FC02460B4600201949FFF7FE
:100CC80009FE78EE687A064617EE900A0F46FFF797
:100CD80083FC02460B4630463946FFF7D1FC0246F4
:100CE8000B4600201049FFF717FBFFF7DBFE2060DB
:100CF800ACE70E4B034CD3ED007A77EEE87AD6E7F3
:100D08003800002030000020C0000020333353405A
:100D180000008039080000202C000020340000204A
:100D2800000000200000084000001C4004000020D3
:100D38002E4B2F4A2F4C304EDFF8C8802F4D80B5F0
:100D48009A6001F057FCFFF7FDFE00F05FF800F035
:100D580057F900F01DF900F037F9294FB3EE018A71
:100D6800FFF762FFD4ED007AF4EEC87AF1EE10FADC
:100D7800F6D5384600224FF4805101F09BFB3846E7
:100D880000224FF4806101F095FB384600224FF4B1
:100D9800807101F08FFB304600224FF4004101F0D2
:100DA80089FB304600224FF4005101F083FB3046A6
:100DB80000224FF4006101F07DFB404600224FF411
:100DC800004101F077FB284600224FF4004101F072
:100DD80071FB284600224FF4005101F06BFB002202
:100DE8004FF40061284601F065FBB7E700ED00E02D
:100DF8000000010830000020000C024000100240F2
:100E08000000024000040240704700BF2DE9F04393
:100E18008BB00024464B00941A6B464DDFF82091A6
:100E2800DFF82081444F454E42F001021A631A6BE5
:100E380002F001020092009A01941A6B42F010022B
:100E48001A631A6B02F010020192019A02941A6B4B
:100E580042F002021A631A6B02F002020292029A2C
:100E680003941A6B42F008021A631A6B02F0080224
:100E78000392039A04941A6B42F004021A631B6BE0
:100E880003F004030493284601224FF47841049B9D
:100E980001F010FB484601224FF4404101F00AFBE3
:100EA800404601224FF47C4101F004FB3846012200
:100EB8004FF4007101F0FEFA012230464FF47C51E4
:100EC80001F0F8FA284605A901254FF4784305935F
:100ED80007940894069501F0D7F9484605A94FF4F8
:100EE8004043059306950794089401F0CDF94046D0
:100EF80005A94FF47C43059306950794089401F0DF
:100F0800C3F9384605A94FF400730593069507946D
:100F1800089401F0B9F94FF47C5305A930460695B9
:100F280007940894059301F0AFF90BB0BDE8F0837E
:100F38000038024000100240000802400000024051
:100F480000040240000C024002680F4B9A4200D095
:100F5800704710B586B0002103F58C3300915A6CA8
:100F68000A4842F480725A645B6C039103F48073FC
:100F780000931022032301A9009C0192029301F01F
:100F880083F906B010BD00BF0020014000000240F8
:100F98000B4B0C4A10B50C211A604FF4E1340022B7
:100FA80018465C6059619A60DA601A619A61DA6180
:100FB80000F0ECFC00B910BDBDE81040FFF724BFFD
:100FC800C0000020004C00400B4B0C4A10B50C210F
:100FD8001A604FF4E134002218465C6059619A6047
:100FE800DA601A619A61DA6100F0D0FC00B910BDCC
:100FF800BDE81040FFF708BF800000200010014046
:101008000B4B0C4A10B50C211A604FF41644002201
:1010180018465C6059619A60DA601A619A61DA610F
:1010280000F0B4FC00B910BDBDE81040FFF7ECBEFD
:101038000001002000440040F0B503683C4A934298
:1010480089B02BD03B4A93424DD03B4A934201D0C2
:1010580009B0F0BD0024394B0294196C384841F4AA
:10106800003119641B6C03F4003302930322072335
:1010780003A9602702260125DDF808E006920793F8
:1010880003970496059501F0FFF82246214626208D
:1010980001F038FA262001F06BFAD9E70024274B33
:1010A8000094196C274841F4002119641B6C03F45F
:1010B800002300930322082303A94FF44067022664
:1010C8000125DDF800E0069207930397049605953D
:1010D80001F0DAF822462146342001F013FA3420D0
:1010E80001F046FAB4E70024144B0194596C1648F1
:1010F80041F0100159645B6C03F010030193032263
:10110800072303A9C02702260125DDF804E006927B
:10111800079303970496059501F0B6F822462146F1
:10112800252001F0EFF9252001F022FA90E700BF11
:10113800004C0040001001400044004000380240CC
:10114800000C02400008024000040240704700BF43
:10115800FEE700BFFEE700BFFEE700BFFEE700BFF7
:10116800704700BF704700BF704700BF08B501F067
:101178005BFABDE8084001F023BA00BF014800F05F
:10118800D7BC00BF80000020014800F0D1BC00BFE0
:1011980000010020014800F0CBBC00BFC0000020C7
:1011A80008B5032001F09CF9002211466FF00B00EE
:1011B80001F0A8F9002211466FF00A0001F0A2F927
:1011C800002211466FF0090001F09CF90022114637
:1011D8006FF0040001F096F9002211466FF0030049
:1011E80001F090F9002211466FF0010001F08AF930
:1011F800002211464FF0FF30BDE8084001F082B9E7
:10120800002800F0AA80F8B5036C04463BB1236CB3
:10121800DB060CD50023012084F83C30F8BD43647C
:1012280080F83C30FFF790FE236CDB06F2D4226C8A
:101238004B4923684B4D22F4885222F0020242F0B7
:10124800020222644A6822F440324A604A686068AE
:1012580002434A6059682069D4F808E0E768A26A3E
:1012680021F4807159605E6846EA00265E605E6817
:1012780026F040765E60586840EA0E00586098682C
:1012880020F4006098609968AA4241EA07019960D1
:1012980046D09968E06A21F07061996099680A43BC
:1012A8009A60996821F0405199609A6802439A605F
:1012B8009968A569206A21F0020199609A6842EA52
:1012C80045029A605A68002833D122F400625A60B5
:1012D800DA6AE569276B666922F47002DA62D86A0D
:1012E800013D40EA0550D862986820F40070986083
:1012F800996841EA47219960996821F48061996069
:101308009A68002042EA86229A606064236C23F07F
:10131800030343F001032364002384F83C30F8BD41
:101328009A6822F070629A609A6822F040529A6035
:10133800BEE742F400625A605A6822F460425A607A
:101348004FF4604191FAA1F1626A5868B1FA81F1EB
:10135800013A8A4002435A60BAE70120704700BF49
:10136800002301400100000F10B490F83C3083B016
:101378000022012B019255D0026893680121DB07F6
:1013880080F83C1014D42A4B2A4C1B689168A4FBA3
:1013980003439B0C03EB430341F00101916001936C
:1013A800019B2BB1019B013B0193019B002BF9D1C0
:1013B8009368DC0731D5036C23F4E06323F0010361
:1013C80043F4807303645368590505D5036C23F40B
:1013D800405343F480530364036C13F480531CBFDD
:1013E800436C23F00603436400246FF02201124B80
:1013F80080F83C4011605B68DB060BD1906810F008
:1014080040500AD1936843F08043936003B05DF87D
:10141800044B7047094B9A42F0D0002003B05DF8A6
:10142800044B7047022003B05DF8044B704700BFBF
:101438000C00002083DE1B430023014000200140F4
:1014480003689A68520502D59B68DB053ED470B5DF
:101458000C46054601F0F0F806462A6801E0601CD3
:1014680025D113689907FAD56FF0120313602B6C16
:1014780043F400732B64936813F0405F15D1AB6994
:101488009BB9D36A13F4700F0CD12B6C23F48073BF
:101498002B64286C10F4805007D12B6C43F00103A7
:1014A8002B6470BD93685B05EFD5002070BD24B137
:1014B80001F0C2F8801B8442CFD22B6C002243F08B
:1014C80004032B6485F83C20032070BD036C0022C4
:1014D80043F02003036480F83C200120704700BFDC
:1014E8000368D86C704700BFF0B590F83C3083B003
:1014F8000022012B019257D00D680123092D2E4699
:1015080080F83C3029D804688B68226905EB450EC1
:10151800072707FA0EF722EA07022261226903FA6F
:101528000EF3134323614B68062B2BD803EB83037D
:10153800626B053B1F21994022EA01026263626BDC
:1015480006FA03F313436363364B9C423ED00023F1
:1015580080F83C30184603B0F0BD04688B68E76833
:10156800AEB206EB46021E3A4FF0070E0EFA02FE26
:1015780027EA0E07E760E76893403B43E3604B6860
:10158800062BD3D90C2B12D803EB8303A3F1230129
:101598001F22236B8A4023EA02032363236B06FA84
:1015A80001F119432163CFE7022003B0F0BD03EB3B
:1015B8008302413AE36A1F21914023EA0103E3626F
:1015C800E36A06FA02F11943E162BDE7122D23D05E
:1015D800A5F11003012BBAD8134A5368102D43F410
:1015E80000035360B3D1114B02F1467202F52E325B
:1015F8001B6802F28332A2FB03239B0C03EB8303D9
:101608005B000193019B002BA1D0019B013B01933F
:10161800019B002BF9D19AE7034A536843F48003EE
:10162800536094E700200140002301400C00002093
:10163800006C70472DE9F047046822698246C0684B
:10164800DAF81C10DAF80830DAF81060DAF8145012
:1016580022F4405202432261E268DAF81800334368
:1016680022F416422B4322F00C020B431343E3608F
:10167800636923F440730343B1F5004F6361AB4BD7
:1016880061D09C4200F0018103F580639C4200F028
:10169800FC8000F0C9FDA64FDAF8043000EB8000AA
:1016A80000EB80009B00B0FBF3F3A7FB03235B096F
:1016B8001D0100F0B9FDDAF8043000EB80009B0052
:1016C80000EB8000B0FBF3F600F0AEFDDAF8042082
:1016D80000EB8000930000EB8000B0FBF3F3A7FB66
:1016E80003234FF064095B0909FB13631B013233C1
:1016F800A7FB03235B0903F0F00600F095FDDAF879
:10170800042000EB8000930000EB8000B0FBF3F8AE
:1017180000F08AFDDAF8043000EB80009B0000EB53
:101728008000B0FBF3F0A7FB0030400909FB1083F1
:101738001B013233A7FB0323C3F3431333432B4467
:10174800A360BDE8F0879C425DD003F580639C42AE
:1017580059D000F069FD764FDAF8043000EB8000CC
:1017680000EB80005B00B0FBF3F3A7FB03235B09EE
:101778001E0100F059FDDAF8043000EB80005B0030
:1017880000EB8000B0FBF3F500F04EFDDAF8042022
:1017980000EB8000530000EB8000B0FBF3F3A7FBE5
:1017A80003235B094FF0640909FB1353DB00323351
:1017B800A7FB03231B0903F4F87500F035FDDAF8DD
:1017C800042000EB800000EB80005300B0FBF3F82E
:1017D80000F02AFDDAF8043000EB800000EB80000E
:1017E8005B00B0FBF3F3A7FB03235B0909FB13833F
:1017F800DB003233A7FB0323C3F3421333442B44E8
:10180800A360BDE8F08700F027FD494FDAF80430FF
:1018180000EB800000EB80005B00B0FBF3F3A7FB5C
:1018280003235B091E0100F017FDDAF8043000EB12
:1018380080005B0000EB8000B0FBF3F500F00CFDCE
:10184800DAF8042000EB8000530000EB8000B0FBC6
:10185800F3F3A7FB03234FF064095B0909FB135358
:10186800DB003233A7FB03231B0903F4F87500F0F0
:10187800F3FCDAF8042000EB8000530000EB800052
:10188800B0FBF3F800F0E8FCA4E700F0E5FC284F13
:10189800DAF8043000EB800000EB80009B00B0FB1E
:1018A800F3F3A7FB03235B091D0100F0D5FCDAF86D
:1018B800043000EB80009B0000EB8000B0FBF3F6E7
:1018C80000F0CAFCDAF8042000EB8000930000EB7B
:1018D8008000B0FBF3F3A7FB03234FF064095B0917
:1018E80009FB13631B013233A7FB03235B0903F0D6
:1018F800F00600F0B1FCDAF8042000EB8000930059
:1019080000EB8000B0FBF3F800F0A6FCDAF8043036
:1019180000EB800000EB80009B00B0FBF3F3A7FB1B
:1019280003235B0909FB138302E700BF0010014092
:101938001F85EB512DE9F04107460E4690461D469E
:101948003C6801E06B1C06D1206836EA0003F9D137
:101958000020BDE8F08135B100F06EFEA0EB080074
:101968008542EDD23C68E36823F4D073E360636991
:10197800202223F0010300216361032087F8392026
:1019880087F8381087F83A20BDE8F08160B338B599
:1019980090F83930044603F0FF0203B32268242389
:1019A80084F83930D36823F40053D3602046FFF716
:1019B80041FE23681A6922F490421A615A6922F09A
:1019C8002A025A61DA680025202142F40052DA60BE
:1019D8002846E56384F8391084F83A1038BD80F851
:1019E8003820FFF729FBD9E7012070472DE9F0439C
:1019F8000F4690F83910202983B003D0022003B095
:101A0800BDE8F083002F3ED0002A3CD0984690F8DD
:101A18003830012B0446F1D0002001212123E06356
:101A280084F8381084F83930019200F005FE019AE4
:101A3800A2848146E28406E0FFF77CFF28BB236886
:101A48003A785A600137E58CADB243464A46802160
:101A58002046E5B1E58CA668013DADB2B6F5805FDC
:101A6800E584E9D143464A4680212046FFF762FFD4
:101A780058B93B8821682269C3F308034B60002AE0
:101A8800E0D10237DFE70120B9E70320B7E74021BB
:101A9800FFF750FF0028F8D1202384F8380084F895
:101AA8003930ACE7704700BF704700BF8368B3F5B3
:101AB800805F28D0036973B10368826A5B68511C30
:101AC80003F07F0381621370C38D013B9BB2C38512
:101AD80043B100207047836A0268591C52688162CA
:101AE8001A70F1E70268D16821F4907110B5D160DD
:101AF8005169202421F00101516180F83A40FFF733
:101B0800D3FF002010BD0269836A3AB9026852689F
:101B1800C2F3080223F8022B8362D5E702685268F1
:101B2800D2B223F8012B8362CEE700BF704700BF13
:101B380003681A6870B51607DD685969044649D004
:101B480011F0010152D0D60705D5E80503D5E06BA1
:101B580040F00100E06356077AD5002900F0848040
:101B6800E16B900741F00201E16376D5E16B41F04A
:101B78000401E163110772D4E16B002929D09106B1
:101B880005D5AA0603D594F83A20222A7CD05D69A7
:101B9800E16B0E0702D415F040057AD0DA6822F41A
:101BA8009072DA605A69202122F001025A6184F8A1
:101BB8003A105A6955065ED55A69606B22F04002A0
:101BC8005A61002857D03B4B036500F077FC00288A
:101BD80055D170BD96060CD5A9060AD590F83A30AD
:101BE800222BF6D1BDE87040FFF760BF15F4907F57
:101BF800A9D110060ED45606EBD56D06E9D5DA68DC
:101C0800202122F04002DA60204684F83910FFF7DC
:101C180049FF70BD2906EED594F83920212AD8D17C
:101C2800A268B2F5805F226A38D0511C216212780E
:101C38005A60E28C013A92B2E284002AC9D1DA6889
:101C480022F08002DA60DA6842F04002DA6070BDA1
:101C580096070BD5002989D18EE711078CD5E16B42
:101C680041F00801E16387E7900785D4100783D521
:101C7800002981D0F3E72046FFF758FF70BD606B5D
:101C8800BDE87040036D18472046FFF70FFF236833
:101C98007DE72046FFF74AFFE56370BD118820699C
:101CA800C1F30801596010B902322262C1E701325A
:101CB8002262BEE7C11C010808B5836B0022DA85E1
:101CC8001846DA84FFF732FF08BD00BFF0B5036895
:101CD800DD0783B004462FD5A3498A6802F00C02B9
:101CE800042A00F0F4808A6802F00C02082A00F046
:101CF800EA806368B3F5803F00F02C81B3F5A02F2C
:101D080000F00081984D2A6822F480322A602A68FF
:101D180022F480222A60002B40F0FD8000F08CFC29
:101D2800064605E000F088FC801B642800F2AA80C3
:101D38002B689B03F6D423689F072DD58A4A9168A0
:101D480011F00C0F00F0A580916801F00C01082932
:101D580000F09B80E368002B00F0EB80834B824D02
:101D680001221A6000F068FC064605E000F064FCF9
:101D7800801B022800F286802B689807F6D5296810
:101D8800F82292FAA2F22369B2FA82F221F0F8015B
:101D980093400B432B6023681A0720D4590734D487
:101DA800A369CBB1704DAA6802F00C02082A77D05B
:101DB800022B6F4B4FF000021A6000F0D18000F048
:101DC8003BFC2C46054604E000F036FC401B02288C
:101DD80058D823689B01F7D4002003B0F0BD63698D
:101DE800002B60D0634B604D01221A6000F024FC88
:101DF800064604E000F020FC801B022842D86B6FE6
:101E08009F07F7D523685907CAD5574B5A4D002263
:101E180001921A6C42F080521A641B6C03F08053D2
:101E28000193019B2B6843F480732B6000F004FC42
:101E3800064604E000F000FC801B022822D82B682C
:101E4800DA05F7D5A368012B00F0F180052B00F027
:101E5800D580454D2A6F22F001022A672A6F22F0A9
:101E680004022A67002B40F0D28000F0E5FB41F223
:101E7800883607462B6F980792D500F0DDFBC01B0C
:101E8800B042F7D9032003B0F0BD526856023FF5BF
:101E980061AF354A1268950723D5E268012A20D038
:101EA800012003B0F0BD334A2F4D136000F0C4FB8E
:101EB800064604E000F0C0FB801B0228E2D86B6FE6
:101EC8009807F7D49EE74A6850027FF512AF264A72
:101ED800126891037FF530AF6268002A7FF42CAF57
:101EE800DEE7214DF821286891FAA1F12269B1FABB
:101EF80081F120F0F8008A4002432A601A077FF532
:101F08004DAF6CE7184B1A6842F480221A601A68C1
:101F180042F480321A6000F08FFB134D064604E04D
:101F280000F08AFB801B6428ACD82B689A03F7D58D
:101F380001E70E4A0C4D136000F07EFB064604E0F4
:101F480000F07AFB801B02289CD82B689907F7D4ED
:101F5800236821E7044A136843F480331360DAE7FF
:101F680000F06AFB06460FE00038024000004742D6
:101F780060004742800E47420070004000F05CFB62
:101F8800801B02283FF67EAF2B689901F6D447F6EE
:101F9800C07696FAA6F64FF44032B6FA86F692FA6A
:101FA800A2F24FF07061B2FA82F091FAA1F1A26A3E
:101FB800676AE369D4F820E0E46A520843EA0E034A
:101FC80007FA06F6013A8240B1FA81F1334304FA7E
:101FD80001F11343194A1A4C0B4301216B6011603C
:101FE80000F02AFB054605E000F026FB401B02280E
:101FF8003FF648AF23689A01F6D5EDE6104B1A6F05
:1020080042F004021A671A6F42F001021A6700F0E0
:1020180013FB0B4D074641F288362B6F9B073FF5A4
:10202800BFAE00F009FBC01BB042F6D92AE7044A4C
:10203800136F43F001031367E9E700BF60004742ED
:1020480000380240194A936803F00C03042B2BD084
:10205800082B27D15168536801F03F0113F4800F12
:10206800536847F6C07292FAA2F0B0FA80F003EA19
:10207800020323FA00F314BF0D480E48B0FBF1F039
:1020880000FB03F0094B4FF440325B6892FAA2F26E
:10209800B2FA82F203F44033D34001335B00B0FB61
:1020A800F3F0704703487047014870470038024012
:1020B80040787D010024F400574A136803F00F03A9
:1020C8008B4208D2CBB21370136803F00F03994206
:1020D80001D00120704703689A072DE9F04106D521
:1020E8004E4C8568A26822F0F0022A43A260DF07FE
:1020F80006460C4626D54268012A00F08780931EC2
:10210800012B464B1B687BD9990728D5434DAB68F3
:1021180023F003031343AB6000F08EFA7368012BBE
:10212800074641F288384FD0022B58D0032B05D1EF
:1021380060E000F081FAC01B404564D8AB6813F03A
:102148000C0FF6D1344A136803F00F039C4209D2EE
:10215800E3B21370136803F00F039C4202D001200E
:10216800BDE8F08133685A0706D52C49F0688A68BB
:1021780022F4E05202438A601B0707D5274A3169D7
:10218800936823F4604343EAC1039360FFF75AFF5F
:10219800224B0146F0229B6892FAA2F2B2FA82F22E
:1021A80003F0F003D3401E481E4AC35C002021FA06
:1021B80003F3136000F008FA0020BDE8F08100F096
:1021C8003BFAC01B40451ED8AB6803F00C03042B38
:1021D800F5D1B7E700F030FAC01B404513D8AB681B
:1021E80003F00C03082BF5D1ACE700F025FAC01B6F
:1021F800404508D8AB6803F00C030C2BF5D1A1E7D8
:10220800980183D4ABE70320BDE8F081034B1B683A
:102218009D033FF57BAFA2E7003C02400038024037
:10222800242701080C000020084B4FF4E0529B685B
:1022380092FAA2F2B2FA82F203F4E053D3400449CC
:10224800044ACB5C1068D840704700BF0038024091
:10225800242701080C000020084B4FF460429B68BB
:1022680092FAA2F2B2FA82F203F46043D34004492C
:10227800044ACB5C1068D840704700BF0038024061
:10228800242701080C0000202DE9F04FD1F800C0E8
:10229800DFF81482DFF814E283B0002503E001358B
:1022A800102D00F09B800123AB4003EA0C029342FF
:1022B800F5D14E6826F0100ABAF1020F00F09180AD
:1022C8004FEA45090324D0F800B004FA09F4E443BE
:1022D80006F003070BEA040B07FA09F70AF1FF3ABD
:1022E80047EA0B07BAF1010F076040F2A080C76800
:1022F8008B683C4003FA09F32343C360F300CED54F
:102308004FF00009CDF80490D8F8443043F48043E6
:10231800C8F84430D8F8444025F0030303F180435B
:1023280004F4804403F59C33019405F00304019FF1
:10233800D3F808A0A4000F27A7402AEA070A544F99
:10234800B84222D007F58067B84200F08380514F29
:10235800B84200F08480504FB84200F085804F4F5B
:10236800B84200F086804E4FB84200F087804D4F4B
:10237800B84200F08880DFF8389148450CBF4FF02C
:1023880007094FF0080909FA04F94AEA09079F60A2
:10239800DEF80030D443F70354BF23401343CEF88C
:1023A8000030DEF80430B70354BF23401343CEF89F
:1023B8000430DEF80830F70254BF23401343CEF848
:1023C8000830DEF80C30B60205F1010554BF234091
:1023D8001343102DCEF80C307FF465AF03B0BDE881
:1023E800F08F4FEAD50900EB890905F00707D9F8FE
:1023F8002040BF004FF00F0B0BFA07FB24EA0B0A33
:102408000C69BC4044EA0A04C9F820404FEA45096F
:102418000324D0F800A004FA09F4E44306F0030703
:102428000AEA040A07FA09F747EA0A070760876809
:1024380007EA040ACF6807FA09F747EA0A07876034
:10244800D0F804A0C6F300172AEA0303AF401F43DD
:1024580047604CE74FF0010909FA04F995E74FF096
:10246800020909FA04F990E74FF0030909FA04F997
:102478008BE74FF0040909FA04F986E74FF00509DC
:1024880009FA04F981E74FF0060909FA04F97CE72B
:102498000000024000080240000C02400010024008
:1024A800001402400018024000380240003C01407D
:1024B800001C024002B909048161704790F8353068
:1024C800022B03D08023436501207047026805234F
:1024D80080F83530136823F001031360002070473B
:1024E800074AD3684FF6FF010B40000243F0BF6371
:1024F80000F4E06043F400330343D360704700BF47
:1025080000ED00E0184B70B4DC68C4F30224C4F199
:102518000706042E04F1040328BF0426062B17D946
:10252800033C0125A540013D2A400123B340013B5E
:102538001940A140002841EA02010CDB00F160408B
:1025480000F561400901C9B280F8001370BC7047FA
:1025580000221446E9E7054B00F00F000901034487
:10256800C9B2197670BC704700ED00E0FCEC00E0E1
:1025780000F01F0101234009024A8B4042F8203035
:10258800704700BF00E100E00138B0F1807F0ED253
:10259800084B10B4084C5860F02084F8230000223F
:1025A800072110469A6019605DF8044B70470120B6
:1025B800704700BF10E000E000ED00E0704700BF8A
:1025C80008B5FFF7FBFF08BD084B094A1B6810B5A3
:1025D800A2FB032304469809FFF7D6FF21460022F1
:1025E8004FF0FF30FFF78EFF002010BD0C000020D9
:1025F800D34D621008B50B4B1A6842F400721A608A
:102608001A6842F480621A601A6842F480721A608A
:102618000320FFF765FF0020FFF7D6FFFEF7C0FD98
:10262800002008BD003C0240024A136801331360D1
:10263800704700BF40010020014B1868704700BF79
:102648004001002010B582B00190FFF7F5FF044665
:10265800FFF7F2FF019B001B9842F9D302B010BDAF
:102668001049114BD1F8882042F4700210B4C1F817
:1026780088201A680D4C002042F001021A60986008
:102688001A6822F0847222F480321A605C601A6838
:102698004FF0006422F480221A60D8608C605DF8E4
:1026A800044B704700ED00E0003802401030002471
:1026B800DFF834D0002103E00C4B5B584350043161
:1026C8000B480C4B42189A42F6D30B4A02E00023FF
:1026D80042F8043B094B9A42F9D3FFF7C1FFFDF7D3
:1026E800A1FDFEF725FB7047000002203C270108EA
:1026F80000000020100000201000002044010020ED
:10270800FEE70000F8B500BFF8BC08BC9E4670475D
:0C271800F8B500BFF8BC08BC9E46704736
:102724000000000001020304010203040607080973
:04273400F5010108A2
:04273800CD010108C6
:10273C009A99793F85EB01400000C03F0024F400DA
:04000005080126B90F
:00000001FF
